:020000040000FA
:020000004E2888
:08000800FD00030EFE000A08D2
:10001000FF000408ED0000308A000B191028332877
:100020000B11AE0F1428AD0A1A302E02031D1F2823
:1000300006302D02031C1F280230B206321535305F
:100040002E02031D33280C302D02031C33280330ED
:10005000B2063215AD01AE01B00F2F28AF0A2C1A2F
:1000600033289F2E3C206D0884007F088A007E0E76
:100070008300FD0E7D0E0900B41F4D285930250266
:10008000031D482857302602031C4828B4164D2863
:1000900026082504031D4D28341708008312850106
:1000A000860187019F01831606309F00003085007E
:1000B00000308600BF308700D130810003178801EF
:1000C00089010313831220308B0053270730C600A9
:1000D0000430C7008A15C0238A11B401B417403018
:1000E0008700203084000630C300031726308D00BF
:1000F000031783160C1483120C088D0A0313C3080C
:10010000031986288000840AC3037828B100A60159
:10011000AD01AE01AC018B17FD200030DA0092304A
:10012000DB00C02850346534723470346534743464
:10013000753461346C342034433461346C34653448
:100140006E3464346134723400345634653472343D
:10015000733469346F346E34203431342E34333494
:10016000303400346234793420346D342E347934B0
:1001700061346D3461346D346F3474346F340034F1
:100180000130D5000130D600B8270430D500033047
:10019000D600B8270430D5000630D600B8271A217B
:1001A00002301321202112218A156F258A11122174
:1001B0001A211221202112211A211221202112217B
:1001C0001A2103301321252102301321A601AD018C
:1001D000AE01AC012C14C001B301B601B7012A294C
:1001E0008316071283128A15D9238A110716033042
:1001F0000A2783160716831208001030C800033040
:10020000C9006430CA000030CB00F0201E300A273D
:100210001730C8000430C9006430CA000030CB0079
:10022000F02008000130C300A60143082602031C89
:10023000152908000130D7008A15D4268A11080034
:10024000D7018A15D4268A1108000330D100030192
:100250004327080037119223B323AB242C1C4C29CD
:100260003F24F7232C10B41E40297030C8000330FF
:10027000C9006430CA000030CB00F020B4124C2911
:10028000341F4C29E030C8000630C900E830CA00ED
:100290000330CB00F0203413AC1D51290A16D823AB
:1002A0000A1284303002031D5A2903302F02031D25
:1002B0005A290713AC1C6E29AC10AC15F625013079
:1002C0002302031D2D29312601302202031D2A2974
:1002D00044262108031D2A294D262A2980218F2101
:1002E00033189C29B318952A3319A42AB3191B2350
:1002F000331A3123B31A8B234023371D2E292A2981
:100300000708BF39BF3AB300031D8829B5018E29FC
:10031000AF01B001B31E0717FA300A270800B71F54
:100320009B29321D9B2932111030B70270303705DE
:10033000031D9B29B713080036187E2A071CA7291E
:1003400064300A27B71B7E2A0130B7067B2A321D8C
:100350007E2A3211B50A07303502031D7E2A2C167B
:10036000B501B714371CB8292521B323AB24F723D3
:100370003F247F22071CBA2964300A27361CC22971
:10038000BD22C429B3223610C001C0177525B3237E
:10039000AB248021B3195A2A3318DC29B31CD22983
:1003A0004D26D529331DC929902620082104031D77
:1003B000C7290130A100C729C00140177525B32303
:1003C000AB248021B319C4293318F429B31CEA29BA
:1003D0004426ED29331DE129812620082104031D2F
:1003E000DF290130A100DF29C001C0167525B32324
:1003F000AB248021B319DC2933180E2AB31C022A3E
:100400003126052A331DF929642601262302031CFF
:10041000F7290319F7290130A300F729C001B323F5
:10042000F72340167525AB248021B319F42933181E
:10043000252AB31C1D2AF625132A331D212A5626E8
:10044000132A321D142A3211132AC001AB24C015FD
:100450007525F7233F248021B3190E2A3318372A34
:10046000B318342A331D2B2A0130B106292AC001C2
:10047000401575253F24F7238021B319252A331809
:10048000492AB31C452ACA263A2A331D3C2AE626A5
:100490003A2AC001C01475253F248021B319372A98
:1004A00033185A2AB31C562AC2264C2A331D4D2A09
:1004B000DC264C2AC001B323401475253F2480213B
:1004C000B319492A33186C2AB31C682ABA265E2A43
:1004D000331D5F2AD2265E2AC722031DAC15C00138
:1004E0002C14AD01AE01B7102C12F030B704371840
:1004F0007B2A75257E2A252137152C1472290A306E
:10050000D500C730D6000230DA008A30DB00B827C9
:10051000D6130800203453344534543420344D3439
:100520004F3444344534203400343718A32A361C61
:10053000B322312601302202031D9F2A3B26C72207
:10054000E522B323AB2474293718B22A361CB32210
:10055000642612302202031DAE2A7026C722E5222D
:10056000B323AB2476292008A7002108A80022087D
:10057000A9002308AA00361408002708A0002808AC
:10058000A1002908A2002A08A300361008002708A5
:100590002002031CE12A031DE32A28082102031C70
:1005A000E12A031DE32A29082202031CE12A031D74
:1005B000E32A2A082302031CE12A031DE32AB601C9
:1005C000E42AB610E42AB61408000230D10007303D
:1005D000D600372705303B273730D40003013F27AB
:1005E000D40BEE2A36080319102BB618FC2A053056
:1005F0003B27FE303F27D6170B30D5005617033068
:10060000DA001130DB00B827D613B61C0C2B2930CA
:100610003B27FE303F27D6171130D500B827D61319
:1006200008007F3444346F3477346E3400345534EA
:1006300070347E34003406302502031C292B5530DB
:100640002502031C302B2C16CA2624080319AC14CF
:100650002A2B2C162C14A501A601AD01AE012C12DB
:100660000800341A3F2B8030B406371C3B2B252161
:10067000B71437152C1440145723C0013416080042
:10068000341E562B321D562B3211B40A0F3034054E
:100690000F3C031D562BE030B405371C542B25218D
:1006A000B71037152C14562BC00157230800DB2533
:1006B00034303B270630D4004008031DFE303F276E
:1006C000D40B5F2B40080319752BB41F6C2B033020
:1006D000DA007630DB00702B0330DA008030DB008C
:1006E0000930D500C730D600B82708005334693424
:1006F00067346E3461346C3420344F346E340034DB
:100700005334693467346E3461346C3420344F347C
:1007100066346634003440308706FA300A27FA30EF
:100720000A27080037189D2B0330DA009E30DB00C3
:100730000030D5004130D600B82708005334753456
:1007400020344D346F3420345434753420345734CD
:1007500065342034543468342034463472342034C0
:100760005334613400343718F02B0130D1000301C9
:10077000372703303B272B30D40003013F27D40B0E
:10078000BD2BD501D601C01FCA2B03303B277F30BC
:100790003F27D617200EF323D50A2008F323D613BC
:1007A000D50A401FD82B0F303B277F303F27D61765
:1007B000210EF323D50A2108F323D613D50A2F30AF
:1007C0006427D50AC01EE92B21303B277F303F2705
:1007D000D617220EF323D50A2208F323D6130800D6
:1007E0000A16002808000F39303864270800371827
:1007F0003C2C0130D1000301372733303B270D302B
:10080000D40003013F27D40B012C0A30D500D601B8
:1008100020306427C0191A2C0930D5006130B11876
:100820007030311C20306427D50A6D30311C2030E7
:100830006427332C0130D1000301372733303B27A5
:100840007F303F270830D500D601D61731182D2C20
:100850000430DA003430DB00312C0430DA00383078
:10086000DB00B827D613080032343434483400345F
:1008700031343234483400340A1625280800371839
:100880008C2C0230D100030137270B303B2731304D
:10089000D40003013F27D40B492C0C30D500D601DE
:1008A000401D572C0B303B277F303F27D617240E97
:1008B000311C622C8F242B0E0F39031D622C20302B
:1008C0006427632CF323D50A2B08311C2408F32357
:1008D000D613D50A3A306427D50AC01C742C1D30B3
:1008E0003B277F303F27D617250EF323D50A25084F
:1008F000F323D613D50A3A306427D50A401C852C39
:100900002F303B277F303F27D617260EF323D50AFB
:100910002608F323D61308000A1666280800B1102B
:100920002408AB002B08031D982C1230AB00AA2C16
:1009300012302B02031CAA2C0319A92CAB000E3079
:100940002B02031CA92C10302B020318A92C0630F3
:10095000AB02B11408003718042D0330D100023067
:10096000D6005608372703013B274030D400030147
:100970003F27D40BB72CD60A07305602031DB12CE3
:100980000130D1005608372703013B273330D4000C
:1009900003013F27D40BC82C07250126BD00423098
:1009A000D6000130BB003C08D500D507D507361866
:1009B000E82C23083B02031DE82C203064274F035A
:1009C0003B27401EE52CB21CE82CFE303F27D617F3
:1009D0003B0E0F39031DEF2C20306427F02CF3233E
:1009E000D50A3B08F323D6133D083B020318032D19
:1009F0003B308400F026BC0A07303C02031CD32C99
:100A0000BC01D60AD32C08000A169B280800013026
:100A1000B900B8010130BC0020082426BE00043013
:100A20003E02031C1B2D031D182D210803191B2D2D
:100A30000430BE020F2D21083902031D232D3E086C
:100A400038020319382D0130BC0765253F18BC0A50
:100A500007303C020318BC0039308400F026A03077
:100A60003902031D1B2DB90138308400F0261B2DDF
:100A70000130BA0022083A020319542D3A082426FC
:100A8000C4005525BC0705308A0002303A02031D18
:100A90004C2D65253F18BC0A07303C020318BC00EA
:100AA0003A308400F0263A2D080005308A004403CD
:100AB0005A3E8200033400340334023403340234D7
:100AC00003340334023403340234BF0139082426CA
:100AD0000339031D742D3908031D732D380824268E
:100AE0000339031D742D3F140800DB25400803194A
:100AF000922D0530DA009330DB004008C500C50DAB
:100B000003188D2DC527CE0005308A00DB0A031996
:100B1000DA0A4E08031D822D7F2D0A30D500C7301A
:100B2000D600B82708005934653461347234203453
:100B30004834693420343F340034593465346134E6
:100B4000723420344C346F3420343F3400344D340C
:100B50006F346E347434683420343F3420340034BD
:100B600054346F3464346134793420343F34003485
:100B70003234343448342F3431343234483420342D
:100B80003F34003448346F347534723420343F3489
:100B900000344D3469346E34753474346534203423
:100BA0003F3400345334653463346F346E3464340A
:100BB00020343F3400340330D10007303727D103CD
:100BC00003013B273C30D4004008031DFE303F2783
:100BD000D40BE72DD1033A303B270630D400400830
:100BE000031DFE303F27D40BF22D080001262302FF
:100BF000031DFD2D0130A300002E23308400F026BC
:100C0000080002302202031D102E2108B90020081E
:100C1000B80065253F1C0E2E2930232E2830232EA8
:100C2000043022020319222E063022020319222E3A
:100C3000093022020319222E113022020319222E1A
:100C40003130232E30300800C500450E0F39C40066
:100C50000310C40DC40DC407C40D45080F39440763
:100C6000080022308400F02613302202031D3A2EA1
:100C70000130A20008004426031C432E4D26031C0D
:100C8000432E0130A100080021308400F026A0305E
:100C90002102031D4C2EA101080020308400F02603
:100CA000A0302002031D552EA0010800A303031D40
:100CB0005C2E0126A300632E23080F390F3C031D71
:100CC000632E0630A3020800A203031D692E123012
:100CD0006E2E0F302202031D6F2E0930A200080075
:100CE0008126210803197A2E99302102031D802EB6
:100CF0009026802E2008031D802E9930A000A10090
:100D00000800A103210A031D882E6630A1028F2E40
:100D100021080F390F3C031D8F2E0630A102080059
:100D2000A003200A031D972E6630A0029E2E2008E5
:100D30000F390F3C031D9E2E0630A00208002630FE
:100D40008400F02660302602031CB82EA601253050
:100D50008400F02660302502031CB82EA501243043
:100D60008400F02624302402031CB82EA401AC1405
:100D70002C14322826308400F02660302602031816
:100D8000A601080025308400F026603025020318F3
:100D9000A501080024308400F02624302402031822
:100DA000A401080026308400F926F9302602031D2C
:100DB000DB2E5930A600080025308400F926F930D2
:100DC0002502031DE52E5930A500080024308400BB
:100DD000F926F9302402031DEF2E2330A400080069
:100DE000800A00080F390A3C031D080006308007FE
:100DF000080000080F390319FF2E80030800800344
:100E00000630800208003430062F6930C100C10B63
:100E1000072F0800C1000030C200000000000000E1
:100E2000000000000000000000000000C20B0D2FB9
:100E3000C10B0B2F08008510521C85125218851605
:100E4000000085110000051251188515D1180516EE
:100E50000000051586000000000005110800D20101
:100E60003F301B270800D201C0381B270800D201E1
:100E7000B8381B270800D20140381B270800D201D0
:100E8000D20A1B270800CE00D301530837270301DD
:100E90003B274030D4004E083F27D40B4B2FD30ABA
:100EA000D31D452F0800051401300A270510013015
:100EB0000A2705140330D1002F27003043270301F0
:100EC0003327030133270800CE00D101D10A55088A
:100ED000CF000A304F02031C6F2FCF00D10A03103E
:100EE000CF0D4F080310CF0DCF07511C792F0430C1
:100EF000CF0756083F3937274F083B274E088A2728
:100F00000301D61B7F30561F882FD4000310540DC9
:100F10003F270800D900D8012030D9025908031012
:100F2000D90DD80D0310D90DD80DD9070318D80A3B
:100F30000030D9070318D80A0830D8070530D30085
:100F4000B427D00007308A00D61FA82F7F30D006E4
:100F5000561FAC2F0310D00D50083F27D90A031994
:100F6000D80AD30BA02F080058088A00590882001D
:100F7000C527CE0007308A00DB0A0319DA0A4E08BB
:100F8000031908006427D50AB82F5A088A005B089D
:020F90008200DD
:1010000000340034003400340034003400344F34F1
:10101000003400340034073400340734003414340E
:101020007F3414347F34143424342A347F342A3403
:10103000123423341334083464346234363449347B
:101040005534223450340034053403340034003431
:1010500000341C342234413400340034413422340E
:101060001C340034143408343E3408341434083446
:1010700008343E34083408340034503430340034FA
:101080000034083408340834083408340034603438
:101090006034003400342034103408340434023412
:1010A0003E345134493445343E34003442347F3484
:1010B00040340034423461345134493446342134AC
:1010C000413445344B3431341834143412347F34C1
:1010D0001034273445344534453439343C344A34AB
:1010E000493449343034013471340934053403341B
:1010F0003634493449344934363406344934493471
:1011000029341E340034363436340034003400348C
:101110005634363400340034083414342234413424
:10112000003414341434143414341434003441347A
:10113000223414340834023401345134093406346E
:1011400032344934793441343E347E3411341134EC
:1011500011347E347F3449344934493436343E3492
:1011600041344134413422347F34413441342234D7
:101170001C347F3449344934493441347F34093490
:101180000934093401343E344134493449347A3421
:101190007F340834083408347F34003441347F34D9
:1011A000413400342034403441343F3401347F34FE
:1011B00008341434223441347F34403440344034D1
:1011C00040347F3402340C3402347F347F340434AE
:1011D000083410347F343E344134413441343E3499
:1011E0007F3409340934093406343E3441345134EF
:1011F00021345E347F34093419342934463446347A
:101200004934493449343134013401347F340134B0
:1012100001343F344034403440343F341F342034B0
:10122000403420341F343F344034383440343F3469
:101230006334143408341434633407340834703499
:10124000083407346134513449344534433400346C
:101250007F344134413400340234043408341034CF
:1012600020340034413441347F34003404340234B7
:101270000134023404344034403440344034403487
:1012800000340134023404340034203454345434EF
:10129000543478347F344834443444343834383423
:1012A00044344434443420343834443444344834AA
:1012B0007F343834543454345434183408347E343D
:1012C0000934013402340C345234523452343E3432
:1012D0007F340834043404347834003444347D34A6
:1012E000403400342034403444343D3400347F34BE
:1012F0001034283444340034003441347F344034D2
:1013000000347C3404341834043478347C340834A5
:101310000434043478343834443444344434383471
:101320007C3414341434143408340834143414342D
:1013300018347C347C34083404340434083448349D
:10134000543454345434203404343F34443440341A
:1013500020343C344034403420347C341C34203439
:10136000403420341C343C344034303440343C3439
:10137000443428341034283444340C345034503439
:1013800050343C344434643454344C3444340034A5
:101390000834363441340034003400347F340034AF
:1013A000003400344134363408340034083408340E
:1013B0002A341C34083408341C342A3408340834E1
:1013C000003400340F3408340834083408340F343F
:1013D000003400342C343234023432342C3444346B
:1013E0003C3404347C34443463345534493441341B
:1013F0004134143414347C341434123444343C34C2
:101400001434143474347C3414341C3414347C3464
:10141000103410345434103410347F347F347F341B
:101420007F347F340F340F340F340F340F340034D3
:10143000003400340034003400340034003400340C
:1014400000340034003400340034003400340034FC
:1014500000340034003400340034003400340034EC
:1014600000340034003400340034003400340034DC
:1014700000340034003400340034003400340034CC
:1014800000340034003400340034003400340034BC
:1014900000340034003400340034003400340034AC
:1014A000003400340034003400340034003400349C
:1014B000003400340034003400340034003400348C
:1014C000003400340034003400340034003400347C
:1014D000003400340034003400340034003400346C
:1014E000003400340034003400340034003400345C
:1014F000003400340034003400340034003400344C
:10150000003400340034003400347034503470340B
:1015100000340034003400340F34013401344034DA
:1015200040347834003400341034203440340034F3
:101530000034003418341834003400340A340A34C7
:101540004A342A341E3404342434343414340C34ED
:1015500020341034783404340034183408344C34D3
:10156000483438344834483478344834483448347B
:10157000283418347C34083408347C340834283453
:101580001834403448344834783440345434543473
:1015900054347C34003418340034583440343834F3
:1015A00008340834083408340834013441343D34F4
:1015B00009340734203410347C34023401340E34BE
:1015C0000234433422341E34423442347E344234B2
:1015D0004234223412340A347F34023442343F34E9
:1015E000023442343E340A340A347F340A340A3432
:1015F00008344634423422341E3404340334423432
:101600003E34043442344234423442347E34023470
:101610004F3422341F3402344A344A3440342034A4
:101620001C344234223412342A34463402343F34D7
:1016300042344A34463406344834403420341E346C
:10164000083446344A3432341E340A344A343E3480
:10165000093408340E3400344E3420341E3404343B
:1016600045343D340534043400347F3408341034B8
:101670000034443424341F340434043440344234B9
:1016800042344234403442342A3412342A34063448
:10169000223412347B341634223400344034203463
:1016A0001F340034783400340234043478343F3446
:1016B00044344434443444340234423442342234D2
:1016C0001E340434023404340834303432340234E6
:1016D0007F340234323402341234223452340E3421
:1016E00000342A342A342A3440343834243422341E
:1016F00020347034403428341034283406340A340A
:101700003E344A344A344A3404347F340434143482
:101710000C344034423442347E3440344A344A3407
:101720004A344A347E3404340534453425341C3478
:101730000F34403420341F3400347C3400347E3481
:10174000803430347E3440342034103408347E34D5
:101750004234423442347E340E3402344234223431
:101760001E344234423440342034183402340434B9
:1017700001340234003407340534073400340034B3
:10178000831203134608E1000130E2004708031901
:10179000CD2BE20D6210FF3EC72B6208E300E20989
:1017A0008030460784006208800584136208800543
:1017B00008008124E830F4000330F500F601F70159
:1017C0008A244808F4004908F500F601F701B62418
:1017D000F30CF20CF10CF00CF313F30CF20CF10C13
:1017E000F00CF313F30CF20CF10CF00CF313700883
:1017F000E4007108E50081244A08F4004B08F50074
:10180000F601F7018A246408F4006508F500F60182
:10181000F7010330003E0319142CF40DF50DF60DFD
:10182000F70D7410FF3E0B2CB6247008E800710809
:10183000E9007208EA007308EB000A30F400003097
:10184000F5006408F0006508F1003F257008E40029
:101850007108E50000307102031D302C0330700266
:101860000318332C0800610884006B08003C031D3A
:10187000432C6A08003C031D432C6908003C031DEF
:10188000432C6808003C03187E2C6308800465081C
:1018900003195A2CE601E70166086702031D522C62
:1018A0006508660203185A2CEC015C25E60A031948
:1018B000E70A4C2C6408EC005C256208800565088A
:1018C0000319722CE601E70166086702031D6A2C02
:1018D000650866020318722CEC015C25E60A031900
:1018E000E70A642C6408EC005C250130E802031C64
:1018F000E902031CEA02031CEB02352C6208800596
:101900000800831203130030F0003230F100F201BE
:10191000F3010800831203132230FC00F801F901DF
:10192000FA01FB01FC030319A62C0310FB0CFA0CB3
:10193000F90CF80CF30CF20CF10CF00C031C922CCB
:10194000FC030319A52CA724962CA72408007408CF
:10195000F80775080318750FF90776080318760F4E
:10196000FA0777080318770FFB07080083120313A1
:10197000FB01FA01F901F801E001730DF80D74089B
:101980001B25F30D0730FC00730D15257408731C1F
:10199000CB2C1B25CC2C2D25F30DFC0BC42C720D50
:1019A00015257408731CD62C1B25D72C2D25F20D5C
:1019B0000730FC00720D15257408721CE12C1B25E4
:1019C000E22C2D25F20DFC0BDA2C710D1525740877
:1019D000721CEC2C1B25ED2C2D25F10D0730FC0085
:1019E000710D15257408711CF72C1B25F82C2D255D
:1019F000F10DFC0BF02C700D15257408711C022DD7
:101A00001B25032D2D25F00D0730FC00700D15252D
:101A10007408701C0D2D1B250E2D2D25F00DFC0BB3
:101A2000062D7018142DA7240800F80DF90DFA0DD5
:101A3000FB0DE00D0800F8027508031C750FF90294
:101A40007608031C760FFA027708031C770FFB0257
:101A50000301031C0130E0020800F80775080318B1
:101A6000750FF90776080318760FFA077708031839
:101A7000770FFB07030103180130E007080083120A
:101A80000313F801F9011030FC00710DF80DF90D88
:101A90007408F8027508031C750FF9020318572D16
:101AA0007408F80775080318750FF9070310F00D8F
:101AB000F10DFC0B452D080083120313EC03EC031E
:101AC0006C08003C0318692DEC03000000000000C6
:101AD000602D0000000000000000000008007425D8
:101AE000A725D625072608000230C3000130CC0008
:101AF000D601D5010130CD003C26551C802D9C26F9
:101B000015270F305505031D7C2DD60A551F7A2D3C
:101B1000CC0A03304C02031D792D0130CC00D601D4
:101B2000D5010130CD006C26551C972DB826152700
:101B30000F305505031D932DD60A551F912DCC0A44
:101B400003304C02031D902DC30B762D080002308C
:101B5000C3000230CC00D6013F30D5000130CD00AB
:101B600054265518B42DB8261527550A0F39031DCC
:101B7000B02DD60A550FAE2DCC0BAC2D0230CC00BB
:101B8000D6013F30D5000130CD0084265518C92D2F
:101B90009C261527550A0F39031DC52DD60A550F4A
:101BA000C32DCC0BC12DC30BA92D08000230C300DF
:101BB0000230CC000730D6003F30D5008030CD0059
:101BC00084265518E42DC6261527550A0F39031DFE
:101BD000E02DD603550FDE2DCC0BDC2D0230CC00D2
:101BE0000730D6003F30D5008030CD005426551840
:101BF000FA2DAA261527550A0F39031DF62DD603EF
:101C0000550FF42DCC0BF22DC30BD82D080002304C
:101C1000C3000130CC000730D600D5018030CD00A4
:101C20006C26551C142EAA2615270F305505031DAA
:101C3000102ED603551F0E2ECC0A03304C02031D66
:101C40000D2E0130CC000730D600D5018030CD00FC
:101C50003C26551C2C2EC62615270F305505031D76
:101C6000282ED603551F262ECC0A03304C02031D06
:101C7000252EC30B092E08004C08D1005508031D62
:101C8000442ECC1C522E4A2E3F305502031D4A2EA4
:101C90004C1C522E5508092703010D270130C31C87
:101CA00003011127D50A08004C08D1003F30550226
:101CB000031D5D2E4C1C6A2E622E5508031D622EDC
:101CC000CC1C6A2E5508092703010D270130C31CBF
:101CD00003011127D50308004C08D1005508031D46
:101CE000742ECC1C822E7A2E3F305502031D7A2E84
:101CF0004C1C822E5508092707300D278030C31C45
:101D000003011127D50A08004C08D1003F305502C5
:101D1000031D8D2E4C1C9A2E922E5508031D922EBB
:101D2000CC1C9A2E5508092707300D278030C31C7C
:101D300003011127D50308000130D1000301092751
:101D400056080D274D08431CA62EFF3A11270314F1
:101D5000CD0D08000130D1000301092756080D27D9
:101D60004D08431CB42EFF3A11270314CD0C080074
:101D70000230D1003F30092756080D274D08431C7B
:101D8000C22EFF3A11270314CD0D08000230D100F6
:101D90003F30092756080D274D08431CD02EFF3A27
:101DA00011270314CD0C08000330D10003010D27C7
:101DB000D501550809270130571C03011127D50A01
:101DC000551FDE2E07300D27D50155080927803015
:101DD000571C03011127D50A551FEA2ED103D6013E
:101DE00056080D273F300927FF30571C03011127E4
:101DF000D60AD61DF02ED103D60156080D270301B1
:101E00000927FF30571C03011127D60AD61DFD2EC6
:101E100008008A113B278A1508008A1137278A157E
:101E200008008A113F278A1508000A308A110A27FC
:041E30008A15080007
:10200000D501D601C01BD617200E2120D50A2008E5
:102010002120D613D50A401BD617210E2120D50A20
:1020200021082120D613D50A2F300D21D50AC01A38
:10203000D617220E2120D50A22082120D6130A12F3
:10204000F22B0F3930380D2108000630D50003304F
:10205000B7180230D6005F20D50A5F20D50A5F206E
:102060000630D500C0194B28311C5D28B1183D2819
:102070001230D800E830D90041281330D800883019
:10208000D90003010D21D50A1330D8004C30D900F6
:1020900003010D215D28D6173230311831300D2162
:1020A000D50A3430311832300D21D50A1230D8001B
:1020B0008430D90003010D21D6130A123E2C5C3066
:1020C000D9001230D80003010D2108000130D500DD
:1020D0000630B7180430D6004019D617240E311C2C
:1020E0007A280A128F240A162B0E0F39031D7A281C
:1020F0005F207B282120D50A2B08311C24082120B1
:10210000D613D50A3A300D21D50AC018D617250E98
:102110002120D50A25082120D613D50A3A300D21D1
:10212000D50A4018D617260E2120D50A26082120C8
:10213000D6130A128E2C0730D500D6012F300D2170
:10214000D50A401AD617230E2120D50A23082120AC
:10215000D6130230D5000330B7180230D6000A1269
:1021600007250A1623080A1224260A16BC07BC03F0
:1021700007303C02031CBE28BC00B8283C08DB002A
:10218000DA010310DB0D5B08DB0DDB07E330DB0757
:102190000318DA0A1030DA070330C300DF20D80052
:1021A000DB0A0319DA0ADF20D900DB0A0319DA0A8D
:1021B00003010D21D50AC30BCE280A12062D5A0899
:1021C0008A005B0882001234AC341334C4341334F4
:1021D0006034123498341334743413346034123449
:1021E000C0341334C434133410341234D43413349C
:1021F00010341234FC341234C03413342434133405
:10220000C4341234703413349C34133438341234DC
:10221000AC341234E8341334B034CE00D101D10AD6
:102220005508CF0005304F02031C1829CF00D10AF2
:102230000310CF0DCF0D4F08CF0DCF07511C222912
:102240000430CF075608D0004E0803193829D900AA
:10225000D8012F30D9020310D90DD90D5908D90D45
:10226000D90DD9076C30D9070318D80A1130D8070F
:102270000230D30050087F3964214F0860210A30B2
:10228000D4000301D01BFF3068215C21CE00113047
:102290008A00D01F4D29FF30CE064E086821D90A8A
:1022A0000319D80AD40B45290301D01BFF3068213C
:1022B000D00AD30B3A29080058088A00590882002E
:1022C0000A123B270A1608000A1237270A160800C6
:1022D0000A123F270A160800003400340034003484
:1022E0008034C034E03470343834183418341C343A
:1022F0000E34073403340134003400340034003425
:10230000F834FC340E3406340634063406340E3405
:10231000FC34F8341F343F3470346034603460343B
:10232000603470343F341F340034003418341C34AB
:10233000FE34FE3400340034003400340034003401
:10234000603460347F347F3460346034003400346F
:1023500018341C340E340634063406348634CE3435
:10236000FC3478346034703478347C346E346734C0
:102370006334613460346034063406340634063421
:102380006634F634FE349E340E3406341834383451
:102390007034603460346034613473343F341E34DC
:1023A0008034C034E034703438341C34FE34FE34AD
:1023B0000034003407340734063406340634063457
:1023C0007F347F34063406347E347E34663466349B
:1023D000663466346634E634C634863418343834A9
:1023E0007034603460346034603470343F341F348F
:1023F000E034F034B8349C348E34863486348634F9
:10240000003400341F343F3471346134613461343A
:10241000613473343F341E340634063406340634D3
:102420008634C634E63476343E341E340034003408
:102430007E347F34033401340034003400340034FB
:102440007834FC34CE348634863486348634CE34C4
:10245000FC3478341E343F34733461346134613475
:10246000613473343F341E347834FC34CE348634D3
:102470008634863486348E34FC34F83400340034A8
:10248000613461346134713439341D340F340734AC
:10249000003400340034703470347034003400344C
:1024A000003400340034003400341C341C341C3438
:1024B000003400340034003400340034003400347C
:1024C000003400340034003400340034003400346C
:1024D000003400340034003400340034003400345C
:1024E000FE34FE348634863486348634863486342C
:1024F000063406347F347F3401340134013401342E
:102500000134013400340034FE34FE34803480342D
:102510008034803480348034FE34FE347F347F3421
:102520000134013401340134013401347F347F3407
:10253000FE34FE341C347834E034E03478341C3417
:10254000FE34FE347F347F340034003401340134EF
:10255000003400347F347F347834FC34CE34863415
:1025600086348634863486340E340C3430347034F9
:102570006134613461346134613473343F341E3406
:102580000634063406340634FE34FE34063406348B
:102590000634063400340034003400347F347F3491
:1025A0000034003400340034FE34FE34003400348F
:1025B0008034803400340034FE34FE340F341F3451
:1025C000703460341F341F34603470341F340F345F
:1025D0000034403460346034603460346034E0345B
:1025E000C034803418343C3466346634663466341F
:1025F000663436347F347F348034C034E034603421
:102600006034E034C0348034FE34FE341F343F3450
:102610007034603460346034613431347F347F34FA
:102620008034C034E0346034603460346034E0348A
:10263000C03480341F343F347634663466346634B4
:102640006634663427340334FE34FE348034C034B8
:10265000E03460346034E034C03480347F347F341C
:102660000134013400340034003400347F347F34CA
:102670000034003460346034E634E634003400342E
:102680000034003400340034603460347F347F34EC
:102690006034603400340034E034E034C0346034FA
:1026A000C0348034E0346034C03480347F347F34CC
:1026B0000034003407340734003400347F347F346E
:1026C000E034E0348034C034E03460346034E034EA
:1026D000C03480347F347F34033401340034003418
:1026E000003400347F347F348034C034E0346034CC
:1026F000603460346034E034C03480341F343F349C
:102700007034603460346034603470343F341F346B
:10271000E034E03460346034603460346034603419
:10272000C03480347F347F340634063406340634B3
:102730000634063403340134E034E0348034C034E9
:10274000E03460346034E034C03480347F347F342B
:1027500001340134003400340034003401340134D5
:1027600060346034FE34FE3460346034003400344D
:1027700000340034003400341F343F34703460348B
:102780006034703438341834E034E03400340034C9
:102790000034003400340034E034E0341F343F347B
:1027A0007034603460347034383418347F347F349B
:1027B000AC11203084000630C300031726308D0092
:1027C00003130008840A03178C0083168C130C155E
:1027D00055308D00AA308D008C148C18ED2B0C1107
:1027E00083128D0A0313C3080319FA2BC30BE12BC1
:0627F0003108E32B080094
:02400E00E223AB
:02401000FF3F70
:1042000043006F0070007900720069006700680069
:1042100074002000280043002900200032003000F4
:10422000310034002D003200300031003900200010
:104230006200790020004D002E00590061006D00E1
:1042400061006D006F0074006F00FF00200014001B
:0A4250001100010000000000000052
:00000001FF
